:1000000012C02CC02BC02AC029C028C027C026C0BF
:1000100025C053C023C022C021C020C01FC01EC0A5
:100020006FC1DBC21BC011241FBECFE5D4E0DEBF11
:10003000CDBF11E0A0E6B0E0E4E4F2E102C005903B
:100040000D92AE36B107D9F711E0AEE6B1E001C0CE
:100050001D92AF37B107E1F702D0F2C8D1CFBED0C1
:1000600006D0B6D2BED0789401D20000FECF81E097
:1000700089BF82E083BF089581E089BF82E083BFAA
:10008000089592B7980F01C0000082B7891B87FDC1
:10009000FBCF089520916E0130916F01280F391F19
:1000A000C901089520916E0130916F01821B930B5D
:1000B00080709078892F90E008951F920F920FB66C
:1000C0000F9211248F939F9380916E0190916F01F5
:1000D000019690936F0180936E019F918F910F9085
:1000E0000FBE0F901F90189590917301992311F4F2
:1000F000AB9A979A80917101981709F4AB98809107
:100100007201981709F49798892F8F5F8093730174
:10011000893C90F110927301909160008091700180
:10012000980F90937001983C11F48FEF03C09923BE
:1001300019F481E0809360009093710160916200F6
:1001400080916100680F60936100683C11F48FEF4B
:1001500003C0662319F481E08093620070E0882771
:1001600077FD8095982F67D52AE939E949E95EE35B
:1001700042D47DD260937201089590916000809185
:100180007001980F90937001983C11F48FEF03C0A9
:10019000992319F481E080936000892F089560917C
:1001A000620080916100680F60936100683C11F407
:1001B0008FEF03C0662319F481E08093620070E042
:1001C000882777FD8095982F36D52AE939E949E9BE
:1001D0005EE311D44CD2DC01CB010895A39A8F9A2F
:1001E000089581B3886381BB12BA87B38E6087BBE1
:1001F00081E388BB1BBC1ABC19BC18BC13BC91E0C2
:100200009FBD81E485BD8EE087BB88B3817F88BBBD
:1002100088E080BF97B99EBD0895209177018091B5
:100220006300821710F4AB9A282F822F90E09BBDB9
:100230008ABD99BD88BD23BD089590917401923007
:1002400041F1933030F4992361F0913009F057C0B7
:1002500014C09430C1F1943040F1953009F04FC092
:1002600042C081EA8FBD81E685BD88E087BB82B34D
:10027000877D82BB949A82E031C081EA8FBD81E69E
:1002800085BD88E087BB82B3877E82BB959A97B98C
:1002900018C081EA8FBD81E685BD84E087BB82B34B
:1002A000877E82BB959A17B81AC081EA8FBD81E616
:1002B00085BD84E087BB82B38F7C82BB939A82E04A
:1002C00087B94098089581EA8FBD81E685BD82E0B7
:1002D00087BB82B38F7C82BB939A81E087B988B158
:1002E000836088B9089581EA8FBD81E685BD82E08B
:1002F00087BB82B3877D82BB949A17B840980895D4
:100300001F920F920FB60F9211242F933F934F938A
:100310005F936F937F938F939F93AF93BF93EF936D
:10032000FF9390E08091740180FF03C0459903C062
:1003300001C0459991509F5F9F30A0F37EDF80916F
:1003400074018F5F809374018091740166E013D70C
:10035000909374018091750190917601019690932C
:10036000760180937501FF91EF91BF91AF919F91BD
:100370008F917F916F915F914F913F912F910F904E
:100380000FBE0F901F9018959F92AF92BF92CF9281
:10039000DF92EF92FF920F931F931092740188B136
:1003A000857F88B988E280937701209163002832A5
:1003B00010F028E201C0AB9A822F90E09BBD8ABD6D
:1003C00099BD88BD23BD39DF2CE2A22E21E0B22EDB
:1003D000C12CD12C9AE0992EEE24FF24870184E6CB
:1003E00050DE0894E11CF11C011D111DEA14FB04F0
:1003F0000C051D05A0F3C601B5012FE030E040E07B
:1004000050E0C5D62095309540955095A20EB31E6C
:10041000C41ED51E89E1A816B104C104D104A0F4FC
:10042000992039F09A9489E1A82EB12CC12CD12CB5
:100430000BC081E01F910F91FF90EF90DF90CF9064
:10044000BF90AF909F900895F8DE809174018F5F08
:10045000809374018091740166E08DD6909374014D
:10046000449BBACF82B3805882BBB6CFDF92EF9263
:10047000FF920F931F932EE088E190E00FB6F8945F
:10048000A89581BD0FBE21BD8AEF90E003DE909359
:100490007C0180937B0111E051E4D52E4EE0E42EE7
:1004A00038E2F32E07E0A89580917801882309F4BB
:1004B000979880917D0190917E01F4DD892B11F058
:1004C00010927A0190917A0180917701981781F0CA
:1004D0009093770120916300291710F0292F01C014
:1004E000AB9A822F90E09BBD8ABD99BD88BD23BD8C
:1004F0009091740180916400891769F084EF91E014
:10050000C9DD90937C0180937B01109378018091E9
:1005100074018093640080917B0190917C01C2DD25
:10052000892BE1F0AB9A88B1857F88B91092780168
:100530001092790180917701882311F0109379014D
:1005400082B3877C82BB1BBC1ABC19BC18BC13BC11
:100550001FBDD5BCE7BA88B3817F88BB8091790184
:10056000882309F4A0CFAB98109279010DDF88237E
:1005700061F1979A1093780188B18C7F88B988B11E
:100580008A6088B9F092770120916300283210F0D8
:1005900028E201C0AB9A822F90E09BBD8ABD99BD35
:1005A00088BD23BD8CE291E075DD90937C01809342
:1005B0007B0101C0000080917B0190917C0172DD84
:1005C000892BC1F3009364006ECF109379016BCF38
:1005D00082E582B985EC86BF08951F920F920FB60F
:1005E0000F9211242F933F934F935F936F937F93B9
:1005F0008F939F93AF93BF93EF93FF9381B190E05D
:10060000887F907080369105B9F0813691051CF491
:10061000892BA9F017C08038910521F0883F9105FA
:1006200089F40DC083B180937A0188EC90E032DDCB
:1006300090937E0180937D0186B7806806C086B75F
:10064000806986BF82E582B985EC86BFFF91EF9114
:10065000BF91AF919F918F917F916F915F914F91DA
:100660003F912F910F900FBE0F901F901895EF9212
:10067000FF920F931F937B018C0120E030E040E05C
:100680005FE4AED288237CF0C801B70120E030E0FF
:1006900040E05FE45ED129D39B01AC0120503040A3
:1006A0004040504805C0C801B7011FD39B01AC01B1
:1006B000B901CA011F910F91FF90EF900895A0E03A
:1006C000B0E0E4E6F3E085C5DC012B01FA019C9182
:1006D000923008F439C1EB018881823008F433C1CB
:1006E000943069F4843009F02FC111969C911197D0
:1006F0008981981709F428C1A5E6B0E025C18430A6
:1007000009F421C18230A9F4923009F01DC19A0187
:10071000AD0188E0EA010990AE01E90109929E016C
:100720008150C1F7E201898111969C9189238183CF
:1007300008C1923009F407C112962D903C9013978E
:10074000EB018A819B811496AD90BD90CD90DC9099
:100750001797EC80FD800E811F819101281B390BBA
:10076000B90137FF04C066277727621B730B60321D
:1007700071050CF061C0121613066CF537014801C3
:10078000062E04C096948794779467940A94D2F7BF
:1007900021E030E040E050E004C0220F331F441F4E
:1007A000551F6A95D2F721503040404050402E21CD
:1007B0003F2140235123211531054105510521F0E9
:1007C00021E030E040E050E079018A01E628F72896
:1007D000082919293CC0232BD1F1260E371E3501DB
:1007E0004601062E04C096948794779467940A94E1
:1007F000D2F721E030E040E050E004C0220F331F88
:10080000441F551F6A95D2F7215030404040504058
:100810002A213B214C215D2121153105410551053E
:1008200021F021E030E040E050E059016A01A628C3
:10083000B728C828D9280BC0821593052CF01C01B5
:10084000AA24BB24650103C0EE24FF24870111966E
:100850009C91D20111968C91981709F445C0992367
:1008600039F0A80197012A193B094C095D0906C016
:10087000A60195012E193F09400B510B57FD08C0E9
:1008800011823382228224833583468357831DC09D
:1008900081E081833382228288279927DC01821BB1
:1008A000930BA40BB50B84839583A683B7830DC0EC
:1008B000220F331F441F551F2483358346835783DC
:1008C000828193810197938382832481358146813C
:1008D0005781DA01C9010197A109B1098F5F9F4FC3
:1008E000AF4FBF4328F30BC0918333822282EA0CBF
:1008F000FB1C0C1D1D1DE482F5820683178383E01B
:100900008083248135814681578157FF1AC0C901F0
:10091000AA2797FDA095BA2F81709070A070B07033
:100920005695479537952795822B932BA42BB52B5E
:1009300084839583A683B783828193810196938371
:100940008283DF0101C0D201CD01CDB7DEB7E2E184
:100950005CC4A0E2B0E0EEEAF4E047C469837A83C5
:100960008B839C832D833E834F835887E9E0EE2E53
:10097000F12CEC0EFD1ECE010196B7012BD38E019A
:100980000F5E1F4FCE010596B80124D38A8991E0EE
:1009900089278A8BC701B801AE01475E5F4F8FDEA2
:1009A00044D2A096E6E03DC4A0E2B0E0E9EDF4E078
:1009B0001CC469837A838B839C832D833E834F83FE
:1009C0005887F9E0EF2EF12CEC0EFD1ECE010196BA
:1009D000B70100D38E010F5E1F4FCE010596B801FF
:1009E000F9D2C701B801AE01475E5F4F68DE1DD284
:1009F000A096E6E016C4A0E2B0E0E0E0F5E0E9C3CE
:100A000069837A838B839C832D833E834F835887AE
:100A1000CE010196BE01675F7F4FDCD2CE01059605
:100A2000BE016F5E7F4FD6D29985923088F089895A
:100A30008230C8F0943019F4823051F404C084300C
:100A400029F4923081F485E690E0C6C0923049F4F2
:100A500020E09A858A89981321E02A87CE01099699
:100A6000BBC0823049F420E09A858A89981321E03E
:100A70002A8BCE014196B0C02D843E844F84588885
:100A80006D887E888F88988CEE24FF248701AA24A5
:100A9000BB24650140E050E060E070E0E0E0F0E0A1
:100AA000C10181709070892BE9F0E60CF71C081DDC
:100AB000191D9A01AB012A0D3B1D4C1D5D1D80E0E7
:100AC00090E0A0E0B0E0E614F7040805190520F472
:100AD00081E090E0A0E0B0E0BA01A901480F591F01
:100AE0006A1F7B1FAA0CBB1CCC1CDD1C97FE08C018
:100AF00081E090E0A0E0B0E0A82AB92ACA2ADB2A67
:100B00003196E032F10549F0660C771C881C991C7F
:100B10005694479437942794C3CFFA85EA892B8952
:100B20003C898B859C85280F391F2E5F3F4F17C04E
:100B3000CA0181709070892B61F016950795F79422
:100B4000E79480E090E0A0E0B0E8E82AF92A0A2BD8
:100B50001B2B76956795579547952F5F3F4F77FDF0
:100B6000E7CF0CC0440F551F661F771F17FD41606C
:100B7000EE0CFF1C001F111F21503040403090E050
:100B8000590790E0690790E4790760F32B8F3C8F59
:100B9000DB01CA018F779070A070B070803491052E
:100BA000A105B10561F447FD0AC0E114F104010596
:100BB000110529F0405C5F4F6F4F7F4F40781A8ED0
:100BC000FE1711F081E08A8F4D8F5E8F6F8F78A3B3
:100BD00083E0898FCE01499628D1A096E2E115C322
:100BE000A8E1B0E0E5EFF5E000C369837A838B8389
:100BF0009C832D833E834F83588789E0E82EF12C18
:100C0000EC0EFD1ECE010196B701E4D18E010F5E00
:100C10001F4FCE010596B801DDD18985823038F0AD
:100C20008989823020F0C701B8014CD201C08FEF12
:100C30006896E6E0F6C2A8E0B0E0E0E2F6E0D2C2F4
:100C40009B01AC0183E08983DA01C9018827B7FDE4
:100C500083959927AA27BB27B82E21153105410571
:100C6000510519F482E0898339C08823A9F0203026
:100C700080E0380780E0480780E8580729F460E002
:100C800070E080E09FEC2EC0EE24FF248701E21A82
:100C9000F30A040B150B02C079018A018EE1C82EFC
:100CA000D12CDC82CB82ED82FE820F831887C801B3
:100CB000B7016CD001971816190684F4082E04C0E9
:100CC000EE0CFF1C001F111F0A94D2F7ED82FE826A
:100CD0000F831887C81AD90ADC82CB82BA82CE0168
:100CE0000196A3D02896E9E099C2ACE0B0E0EAE72B
:100CF000F6E07FC269837A838B839C83CE01019661
:100D0000BE016B5F7F4F66D18D81823061F1823091
:100D100050F1843021F48E81882351F12EC02F812F
:100D2000388537FD20C06E812F3131051CF06623D8
:100D3000F9F023C08EE190E0821B930B29853A8560
:100D40004B855C8504C056954795379527958A95C0
:100D5000D2F76623B1F050954095309521953F4FDD
:100D60004F4F5F4F0EC020E030E040E050E009C040
:100D70002FEF3FEF4FEF5FE704C020E030E040E0AF
:100D800050E8B901CA012C96E2E04FC2EF92FF92FF
:100D90000F931F937B018C0180E0E81680E0F8063A
:100DA00081E0080780E0180788F48FEFE816F10467
:100DB0000105110531F028F088E090E0A0E0B0E0F6
:100DC00017C080E090E0A0E0B0E012C080E0E8163C
:100DD00080E0F80680E0080781E0180728F088E145
:100DE00090E0A0E0B0E004C080E190E0A0E0B0E0DE
:100DF00020E230E040E050E0281B390B4A0B5B0B4F
:100E000004C016950795F794E7948A95D2F7F701F1
:100E1000E359FF4F8081281B310941095109C9015C
:100E20001F910F91FF90EF900895DF92EF92FF9244
:100E30000F931F93FC01E480F58006811781D18018
:100E40008081823048F480E090E0A0E1B0E0E82AC0
:100E5000F92A0A2B1B2BA5C0843009F49FC08230CD
:100E600021F4EE24FF24870105C0E114F1040105FB
:100E7000110519F4E0E0F0E096C0628173819FEF04
:100E8000623879070CF05BC022E83FEF261B370B76
:100E90002A3131052CF020E030E040E050E02AC05B
:100EA000B801A701022E04C076956795579547951E
:100EB0000A94D2F781E090E0A0E0B0E004C0880F8F
:100EC000991FAA1FBB1F2A95D2F70197A109B10943
:100ED0008E219F21A023B1230097A105B10521F008
:100EE00081E090E0A0E0B0E09A01AB01282B392B23
:100EF0004A2B5B2BDA01C9018F779070A070B0701C
:100F000080349105A105B10539F427FF09C0205CA3
:100F10003F4F4F4F5F4F04C0215C3F4F4F4F5F4FDC
:100F2000E0E0F0E02030A0E03A07A0E04A07A0E4CB
:100F30005A0710F0E1E0F0E079018A0127C060383B
:100F4000710564F5FB01E158FF4FD801C7018F77A8
:100F50009070A070B07080349105A105B10539F48E
:100F6000E7FE0DC080E490E0A0E0B0E004C08FE3B5
:100F700090E0A0E0B0E0E80EF91E0A1F1B1F17FF6B
:100F800005C016950795F794E794319687E0169576
:100F90000795F794E7948A95D1F705C0EE24FF24CE
:100FA0008701EFEFF0E06E2F679566276795902F2A
:100FB0009F77D794DD24D7948E2F8695492F462B83
:100FC000582F5D29B701CA011F910F91FF90EF9033
:100FD000DF900895FC01DB01408151812281622F65
:100FE0006F7770E0221F2227221F9381892F880F9D
:100FF000822B282F30E0991F9927991F11969C93D7
:10100000119721153105A9F54115510561057105A6
:1010100011F482E037C082E89FEF13969C938E9381
:1010200012979A01AB0167E0220F331F441F551F2F
:101030006A95D1F783E08C930DC0220F331F441FB4
:10104000551F12968D919C911397019713969C931F
:101050008E931297203080E0380780E0480780E4C4
:10106000580758F314962D933D934D935C9317971F
:1010700008952F3F310579F441155105610571053A
:1010800019F484E08C93089564FF03C081E08C938D
:1010900012C01C9210C02F57304013963C932E93D1
:1010A000129783E08C9387E0440F551F661F771FCC
:1010B0008A95D1F7706414964D935D936D937C93EC
:1010C000179708951F93DC01FB019C91923008F45F
:1010D00047C08081823008F443C0943051F41196A7
:1010E0001C91843099F58181682F70E0611B710932
:1010F0003FC0843021F0923031F48230B9F18181E7
:10110000882389F12DC011961C9111978230F1F03E
:1011100081811817D9F412962D913C9113978281F1
:1011200093818217930794F028173907BCF014961F
:101130008D919D910D90BC91A02D2481358146818A
:101140005781281739074A075B0718F4112341F024
:101150000AC082179307A407B50740F4112319F0BA
:1011600061E070E005C06FEF7FEF02C060E070E00B
:10117000CB011F910895991B79E004C0991F961720
:1011800008F0961B881F7A95C9F780950895A1E20B
:101190001A2EAA1BBB1BFD010DC0AA1FBB1FEE1FF1
:1011A000FF1FA217B307E407F50720F0A21BB30B3C
:1011B000E40BF50B661F771F881F991F1A9469F7B8
:1011C00060957095809590959B01AC01BD01CF0114
:1011D00008952F923F924F925F926F927F928F92DB
:1011E0009F92AF92BF92CF92DF92EF92FF920F93B6
:1011F0001F93CF93DF93CDB7DEB7CA1BDB0B0FB6C0
:10120000F894DEBF0FBECDBF09942A88398848887C
:101210005F846E847D848C849B84AA84B984C88412
:10122000DF80EE80FD800C811B81AA81B981CE0F09
:10123000D11D0FB6F894DEBF0FBECDBFED010895EE
:04124000F894FFCF50
:1012440001C8FFFF070000000000000000000102C9
:10125400020303030304040404040404040505054D
:101264000505050505050505050505050506060627
:10127400060606060606060606060606060606060A
:1012840006060606060606060606060606070707F7
:1012940007070707070707070707070707070707DA
:1012A40007070707070707070707070707070707CA
:1012B40007070707070707070707070707070707BA
:1012C40007070707070707070707070707080808A7
:1012D400080808080808080808080808080808088A
:1012E400080808080808080808080808080808087A
:1012F400080808080808080808080808080808086A
:101304000808080808080808080808080808080859
:101314000808080808080808080808080808080849
:101324000808080808080808080808080808080839
:101334000808080808080808080808080808080829
:0E134400080808080808080808080808080033
:00000001FF
